:100000000C94F5000C9400000C9400000C9400007B
:100010000C9400000C9400000C9400000C94000060
:100020000C9400000C9400000C9400000C94000050
:100030000C9400000C9400000C9400000C94000040
:100040000C942D010C9400000C9400000C94000002
:100050000C9400000C9441010C9400000C940000DE
:100060000C9400000C9400001818181818181800A8
:1000700003030303030303001B1B1B1B1B1B1B00AE
:1000800000000000001818000000181818181800C8
:100090001B1B1B1B1B1B1B0015150E04040404005B
:1000A0001B1B1B1B1B1B1B000100E80300000000A7
:1000B000000000005D025452582054454136323051
:1000C00030762E30336100726164696F7275626BD5
:1000D000612E61742E7561002054525820544541A0
:1000E00036323030762E303361002020466972730C
:1000F0007420537461727420202000202020204935
:1001000046205365747570202020200044445320FD
:10011000512E2047656E2053657475700049462046
:100120003D200020487A0045646974200020312079
:100130006B487A003130206B487A003130302048EB
:100140007A003530206B487A003120206B487A00E5
:1001500031302020487A0031202020487A002020A9
:100160004B6F656666205665726966792020002EA1
:1001700000414D200035303020487A0052002030B8
:1001800020202020487A0041200030666620002D83
:10019000313020002D323020002D3330200020203F
:1001A000202020002020202020200020202020208F
:1001B0002020002020202020202020005B54585D9B
:1001C000000080C001002D4E414E00494E46000007
:1001D00001003103A8000C000300AA0002003B0349
:1001E000C20101004203C4010000F894EE27EFBBF6
:1001F000F1E0F5BFE5BFF8E1A895A4B7A77FA4BFDC
:10020000F0936000E09360008DE0A2E0BB27ED93E7
:100210008A95E9F780E098E0A0E0B1E0ED930197DE
:10022000E9F7E0EDF1E085919591009761F0A591F6
:10023000B59105901590BF01F00105900D920197C1
:10024000E1F7FB01F0CFE0ECEEBBEFEFEDBFE8E054
:10025000EEBFC0E0D3E00C94D801EA93FA93EFB775
:10026000EA93E0910C03F0910D033196E0930C03B7
:10027000F0930D03E0E0E6BDE991EFBFF991E9915C
:1002800018951A930A930091780010917900B02E76
:10029000C12EF79A0991199118951A930A93EA8138
:1002A000EE0FEE0FEE0FE0640E2F10E0183070F43A
:1002B0000A930395EC81FD813196EC83FD833197A0
:1002C000E491EA930E94850B1F5FF0CF19810881AA
:1002D00025960895E0E0E0932E03E0932F03089520
:1002E0001A9310E0339B11E0349B1260E0912E03CF
:1002F000E11711F40C94D601A0912E03A33021F440
:10030000E0912F03E11709F44BC0123031F5F09959
:1003100017C0E32DF42DA0910003B091010380914B
:10032000020390910303662777270E94DF0DE09375
:100330000003F093010360930203709303030BC067
:10034000E7E8F3E17E168F063CF4E72DF82DEC5933
:10035000FF4F7E2E8F2EF69A23C0F09917C0E32D03
:10036000F42DA0910003B0910103809102039091BC
:100370000303662777270E94E90DA0930003B0933B
:100380000103809302039093030309C0E9E7FCEEA5
:10039000E715F8052CF4E4E6F0E07E1A8F0AF69AE9
:1003A000E0912E03E0932F0310932E0319910895EB
:1003B000E0E8E0936100E0E0E0936100E5B9E0E3AC
:1003C000E4B9E0E0E8B9E4E0E7B9E0E0EBB9EFE098
:1003D000EAB9E0E0E4BDE5E0E5BDE0E0E6BDE7BDAB
:1003E000E8BDE0938000E0938100E0938500E09316
:1003F0008400E0938700E0938600E0938900E09317
:100400008800E0938B00E0938A00E093B600E093CD
:10041000B000E093B100E093B200E093B300E0934A
:10042000B400E0936900EDBBE0936800E1E0E09385
:100430006E00E0E0E0936F00E0937000E093C10095
:10044000E0E8E0BFE0E0E0937B00E0937F00E09332
:100450007E00E0ECE0937C00EBE8E0937A00E0E0E3
:10046000ECBDE093BC00E0E1EA930E94F90BE8E602
:10047000F0E0FA93EA93E0E0EA930FDFE0E7F0E0E0
:10048000FA93EA93E1E0EA9308DFE8E7F0E0FA9311
:10049000EA93E2E0EA9301DFE0E8F0E0FA93EA931E
:1004A000E3E0EA93FADEE8E8F0E0FA93EA93E4E0C6
:1004B000EA93F3DEE0E9F0E0FA93EA93E5E0EA9309
:1004C000ECDEE0EAF0E0FA93EA93E6E0EA93E5DEB8
:1004D000E8E9F0E0FA93EA93E7E0EA93DEDEA0E0F1
:1004E000B0E00E947F0EE530C1F4E0E0EA93EA93C9
:1004F0000E948E0BE6EBF0E0FA93EA930E94E80B81
:10050000E0E0EA93E1E0EA930E948E0BE7ECF0E092
:10051000FA93EA930E94E80B44C0E0E0EA93EA937E
:100520000E948E0BE8EDF0E0FA93EA930E94E80B4C
:10053000E0E0EA93E1E0EA930E948E0BEAEEF0E05D
:10054000FA93EA930E94E80BADE0B0E0E0EFF3EB42
:100550006AE170E00E948B0EA1E0B0E0E0EEF4E40E
:1005600063EA70E00E948B0EA9E0B0E0E0E4F9E5F8
:1005700063E777E00E948B0EA9E0B0E00E94770E5F
:100580000E941E0DA0E0B0E080E89FE40E949A0D5A
:10059000A5E0B0E00E948B0EA0E0B0E0E5E00E9494
:1005A0009B0E1A9919C0F19AE0E0EA93EA930E942F
:1005B0008E0BE8EDF0E0FA93EA930E94E80BE0E09E
:1005C000EA93E1E0EA930E948E0BEBEFF0E0FA93FE
:1005D000EA930E94E80B01C0F198199919C0F39AA7
:1005E000E0E0EA93EA930E948E0BE8EDF0E0FA93E4
:1005F000EA930E94E80BE0E0EA93E1E0EA930E94CC
:100600008E0BECE0F1E0FA93EA930E94E80B01C054
:10061000F39860DEE0917C00EE7FE0937C00E09157
:100620007C00ED7FE0937C00E0917C00EB7FE09329
:100630007C00E0917C00E77FE0937C00E0EDF7E058
:10064000FA93EA930E94AC0C589A58980E949F0B18
:10065000F19BBEC0F2990DC0A1E0B0E00E94770E00
:10066000E0930003F093010360930203709303038C
:10067000F29AF69B2BC00E949F0BE0E0EA93EA936C
:100680000E948E0BEDE1F1E0FA93EA930E94E80BF1
:10069000E0910003F0910103609102037091030364
:1006A0000E94600EE4E1F3E0FA93EA930E943E0CAC
:1006B000E4E1F3E0FA93EA930E94DB0BE3E2F1E07A
:1006C000FA93EA930E94E80BF698F79AF79B39C0E1
:1006D000E0E0EA93E1E0EA930E948E0BE7E2F1E0CA
:1006E000FA93EA930E94E80BE8EEF3E0E315F405D1
:1006F00031F4EDE2F1E0FA93EA930E94E80BE0E1D5
:10070000F7E2E315F40531F4E4E3F1E0FA93EA9358
:100710000E94E80BE4E6F0E0E315F40531F4EBE3C6
:10072000F1E0FA93EA930E94E80BE0E5F3ECE315BD
:10073000F40531F4E2E4F1E0FA93EA930E94E80B65
:10074000F798CEDD1B9926C0E32DF42DE436A0E00A
:10075000FA0719F4E8EEF3E014C0E83EA3E0FA0764
:1007600019F4E0E1F7E20DC0E031A7E2FA0719F46D
:10077000E0E5F3EC06C0E035A3ECFA0759F4E4E653
:10078000F0E03E2E4F2EF79AECE2F1E0FA93EA9376
:100790000E94AC0C19991BC0E0910003F091010379
:1007A0006091020370910303A1E0B0E00E948B0E00
:1007B000F69AF79AE8EEF3E03E2E4F2E0E949F0B3A
:1007C000E8EEF3E0FA93EA930E94AC0CF19840CF84
:1007D000F39B1CC1F4990DC0A9E0B0E00E94770E14
:1007E000E0930003F093010360930203709303030B
:1007F000F49AF69B28C0E0E0EA93EA930E948E0BFD
:10080000EEE1F1E0FA93EA930E94E80BE091000335
:10081000F091010360910203709103030E94600E46
:10082000E4E1F3E0FA93EA930E943E0CE4E1F3E0A2
:10083000FA93EA930E94DB0BE3E2F1E0FA93EA9386
:100840000E94E80BF698F79B39C0E0E0EA93E1E0FC
:10085000EA930E948E0BE7E2F1E0FA93EA930E949A
:10086000E80BE8EEF3E0E315F40531F4E9E4F1E038
:10087000FA93EA930E94E80BE4E6F0E0E315F4054E
:1008800031F4EBE3F1E0FA93EA930E94E80BEAE03B
:10089000F0E0E315F40531F4E0E5F1E0FA93EA93D2
:1008A0000E94E80BE1E0F0E0E315F40531F4E7E540
:1008B000F1E0FA93EA930E94E80BF79811DD1B9997
:1008C00026C0E32DF42DE436A0E0FA0719F4E8EE93
:1008D000F3E014C0E83EA3E0FA0719F4E1E0F0E029
:1008E0000DC0E130A0E0FA0719F4EAE0F0E006C03C
:1008F000EA30A0E0FA0759F4E4E6F0E03E2E4F2E8D
:10090000F79AECE2F1E0FA93EA930E94AC0C1A99A0
:100910007CC0E0910003F0910103609102037091AB
:100920000303A9E0B0E00E948B0EE4E6F0E0FA9346
:10093000EA930E94AC0CA9E0B0E00E94770E0E94FE
:100940001E0DA0E0B0E080E89FE40E949A0DA5E0B3
:10095000B0E00E948B0EE4E6F0E0FA93EA930E9486
:10096000AC0C0E949F0BE0E0EA93EA930E948E0B8E
:10097000EEE5F1E0FA93EA930E94E80BA5E0B0E01F
:100980000E94770EA0E0B0E080E89FE40E949A0DFC
:10099000A0E0B3E00E94E50C0E945B0EE091000332
:1009A000F091010360910203709103030E94600EB5
:1009B000E4E1F3E0FA93EA930E943E0CE0E0EA936C
:1009C000E1E0EA930E948E0BE7EFF0E0FA93EA93FE
:1009D0000E94E80BE4E1F3E0FA93EA930E94DB0B58
:1009E000E8EBFBE0FA93EA930E94AC0CF69AF79AD4
:1009F000E8EEF3E03E2E4F2E0E949F0BE8EEF3E070
:100A0000FA93EA930E94AC0CF398E2CEA5E0B0E032
:100A10000E94770EE0933703F09338036093390315
:100A200070933A03A1E0B0E00E94770EE0930803D0
:100A3000F093090360930A0370930B03ADE0B0E0F9
:100A40000E94770EE0930003F0930103609302038A
:100A5000709303037894F69B2BC1E0E0EA93EA934A
:100A60000E948E0BA0910003B091010380910203BC
:100A700090910303E8EEF3E060E070E00E94320E34
:100A8000E0932A03F0932B03A0910003B09101039C
:100A90008091020390910303E8EEF3E060E070E0E0
:100AA0000E94570EDF01CB01E4E6F0E060E070E069
:100AB0000E94320EE0932C03F0932D03E0912A0361
:100AC000F0912B030E94FE0D0E94600EE4E1F3E022
:100AD000FA93EA930E943E0CE0912C03F0912D03CF
:100AE0000E94FE0D0E94600EE4E2F3E0FA93EA93A6
:100AF0000E943E0CE4E1F3E0FA93EA930E94DB0BE0
:100B0000EFE6F1E0FA93EA930E94E80BE4E2F3E007
:100B1000FA93EA930E94DB0BE9EFF0E0FA93EA9391
:100B20000E94E80BF09935C0E1E7F1E0FA93EA930F
:100B30000E94E80BE8EEF3E0E315F40531F4EDE292
:100B4000F1E0FA93EA930E94E80BE0E1F7E2E315A3
:100B5000F40531F4E4E3F1E0FA93EA930E94E80B40
:100B6000E4E6F0E0E315F40531F4EBE3F1E0FA93A9
:100B7000EA930E94E80BE4EFF1E0E315F40531F4A9
:100B8000E5E7F1E0FA93EA930E94E80BE6ECF0E087
:100B900087C0ECE7F1E0FA93EA930E94E80BE72DB7
:100BA000F82D0E94FE0D0E94600EEEE0F3E0FA9335
:100BB000EA930E943E0C072C082831F4EEE7F1E09E
:100BC000FA93EA930E94E80BA72DB82DE0E0F0E03D
:100BD0000E941A0E0E2EE7EEF3E00E94080EE021AE
:100BE00091F0E9EFF0E0FA93EA930E94E80BEEE06F
:100BF000F3E0FA93EA930E94DB0BE2E5F1E0FA936B
:100C0000EA930E94E80BA72DB82DE8EEF3E00E94CE
:100C10000E0E0E2EEFE0F7E20E94080EE02191F09A
:100C2000E9EFF0E0FA93EA930E94E80BEEE0F3E0DC
:100C3000FA93EA930E94DB0BE3E2F1E0FA93EA9382
:100C40000E94E80BA72DB82DE0E0F0E00E94140E02
:100C50000E2EE9E1FCEF0E940E0EE02161F0EEE0C5
:100C6000F3E0FA93EA930E94DB0BE2E5F1E0FA93FA
:100C7000EA930E94E80BA72DB82DE8E1FCEF0E9453
:100C8000080E0E2EE1EFF8ED0E941A0EE02161F041
:100C9000EEE0F3E0FA93EA930E94DB0BE3E2F1E08B
:100CA000FA93EA930E94E80BF698E1E0E0933103AF
:100CB000F79BBFC3F5997BC3E0E0EA93E1E0EA93D9
:100CC0000E948E0BE7E8F1E0FA93EA930E94E80BAA
:100CD000662031F4EAE8F1E0FA93EA930E94E80B27
:100CE000EAE0E61531F4EFE8F1E0FA93EA930E94C6
:100CF000E80BE4E1E61531F4E4E9F1E0FA93EA9374
:100D00000E94E80BEEE1E61531F4E9E9F1E0FA932F
:100D1000EA930E94E80B9B2CAC2CED2DFE2DEF5B93
:100D2000FE4FE915FA0540F5E7E0EA930E94BA0B99
:100D3000E2E0EA930E94BA0BE2E0EA930E94BA0B67
:100D4000E2E0EA930E94BA0BE2E0EA930E94BA0B57
:100D5000E2E0EA930E94BA0BE2E0EA930E94BA0B47
:100D6000E2E0EA930E94BA0BE2E0EA930E94BA0B37
:100D7000E2E0EA930E94BA0BED2DFE2DEE5EFE4FEF
:100D8000A92DBA2D0E942C0E0E2EED2DFE2DEF5BFF
:100D9000FE4F0E94260EE02141F1E7E0EA930E9417
:100DA000BA0BE2E0EA930E94BA0BE2E0EA930E94F7
:100DB000BA0BE2E0EA930E94BA0BE2E0EA930E94E7
:100DC000BA0BE2E0EA930E94BA0BE2E0EA930E94D7
:100DD000BA0BE2E0EA930E94BA0BE2E0EA930E94C7
:100DE000BA0BE0E0EA930E94BA0BED2DFE2DE35121
:100DF000FF4FA92DBA2D0E942C0E0E2EED2DFE2D8B
:100E0000EE5EFE4F0E94260EE02151F1E7E0EA93EC
:100E10000E94BA0BE2E0EA930E94BA0BE2E0EA9386
:100E20000E94BA0BE2E0EA930E94BA0BE2E0EA9376
:100E30000E94BA0BE2E0EA930E94BA0BE2E0EA9366
:100E40000E94BA0BE2E0EA930E94BA0BE2E0EA9356
:100E50000E94BA0BE9EFF0E0FA93EA930E94E80BE4
:100E6000ED2DFE2DE153FF4FA92DBA2D0E942C0E22
:100E70000E2EED2DFE2DE351FF4F0E94260EE02198
:100E800051F1E7E0EA930E94BA0BE2E0EA930E9494
:100E9000BA0BE2E0EA930E94BA0BE2E0EA930E9406
:100EA000BA0BE2E0EA930E94BA0BE2E0EA930E94F6
:100EB000BA0BE2E0EA930E94BA0BE2E0EA930E94E6
:100EC000BA0BE0E0EA930E94BA0BE9EFF0E0FA9384
:100ED000EA930E94E80BED2DFE2DEB54FF4FA92D58
:100EE000BA2D0E942C0E0E2EED2DFE2DE153FF4F3C
:100EF0000E94260EE02131F1E7E0EA930E94BA0B4E
:100F0000E2E0EA930E94BA0BE2E0EA930E94BA0B95
:100F1000E2E0EA930E94BA0BE2E0EA930E94BA0B85
:100F2000E2E0EA930E94BA0BE2E0EA930E94BA0B75
:100F3000E2E0EA930E94BA0BE8EFF0E0FA93EA935A
:100F40000E94E80BED2DFE2DE156FF4FA92DBA2D85
:100F50000E942C0E0E2EED2DFE2DEB54FF4F0E9405
:100F6000260EE02131F1E7E0EA930E94BA0BE2E0BD
:100F7000EA930E94BA0BE2E0EA930E94BA0BE2E025
:100F8000EA930E94BA0BE2E0EA930E94BA0BE2E015
:100F9000EA930E94BA0BE2E0EA930E94BA0BE0E007
:100FA000EA930E94BA0BE8EFF0E0FA93EA930E940A
:100FB000E80BED2DFE2DE457FF4FA92DBA2D0E9411
:100FC0002C0E0E2EED2DFE2DE156FF4F0E94260E0B
:100FD000E02111F1E7E0EA930E94BA0BE2E0EA9324
:100FE0000E94BA0BE2E0EA930E94BA0BE2E0EA93B5
:100FF0000E94BA0BE2E0EA930E94BA0BE2E0EA93A5
:101000000E94BA0BE2E0EA930E94BA0BE7EFF0E02D
:10101000FA93EA930E94E80BED2DFE2DE658FF4F60
:10102000A92DBA2D0E942C0E0E2EED2DFE2DE4576B
:10103000FF4F0E94260EE02111F1E7E0EA930E94A3
:10104000BA0BE2E0EA930E94BA0BE2E0EA930E9454
:10105000BA0BE2E0EA930E94BA0BE2E0EA930E9444
:10106000BA0BE2E0EA930E94BA0BE0E0EA930E9436
:10107000BA0BE7EFF0E0FA93EA930E94E80BED2D4C
:10108000FE2DE559FF4FA92DBA2D0E942C0E0E2ED4
:10109000ED2DFE2DE658FF4F0E94260EE021F1F0C7
:1010A000E7E0EA930E94BA0BE2E0EA930E94BA0BEF
:1010B000E2E0EA930E94BA0BE2E0EA930E94BA0BE4
:1010C000E2E0EA930E94BA0BE2E0EA930E94BA0BD4
:1010D000E7E0F1E0FA93EA930E94E80BED2DFE2D94
:1010E000E45AFF4FA92DBA2D0E942C0E0E2EED2D85
:1010F000FE2DE559FF4F0E94260EE021F1F0E7E0BA
:10110000EA930E94BA0BE2E0EA930E94BA0BE2E093
:10111000EA930E94BA0BE2E0EA930E94BA0BE2E083
:10112000EA930E94BA0BE0E0EA930E94BA0BE7E070
:10113000F1E0FA93EA930E94E80BED2DFE2DE15BBE
:10114000FF4FA92DBA2D0E942C0E0E2EED2DFE2D37
:10115000E45AFF4F0E94260EE021D1F0E7E0EA9327
:101160000E94BA0BE2E0EA930E94BA0BE2E0EA9333
:101170000E94BA0BE2E0EA930E94BA0BE2E0EA9323
:101180000E94BA0BEEE9F1E0FA93EA930E94E80BB1
:10119000ED2DFE2DED5BFF4FA92DBA2D0E942C0EDB
:1011A0000E2EED2DFE2DE15BFF4F0E94260EE0215D
:1011B000D1F0E7E0EA930E94BA0BE2E0EA930E94E2
:1011C000BA0BE2E0EA930E94BA0BE2E0EA930E94D3
:1011D000BA0BE0E0EA930E94BA0BEEE9F1E0FA9371
:1011E000EA930E94E80BED2DFE2DF896A92DBA2D5D
:1011F0000E942C0E0E2EED2DFE2DED5BFF4F0E945A
:10120000260EE021B1F0E7E0EA930E94BA0BE2E09B
:10121000EA930E94BA0BE2E0EA930E94BA0BE2E082
:10122000EA930E94BA0BE4EAF1E0FA93EA930E948F
:10123000E80BED2DFE2DBD96A92DBA2D0E942C0E8A
:101240000E2EED2DFE2DF8960E94260EE021B1F017
:10125000E7E0EA930E94BA0BE2E0EA930E94BA0B3D
:10126000E2E0EA930E94BA0BE0E0EA930E94BA0B34
:10127000E4EAF1E0FA93EA930E94E80BED2DFE2DEB
:10128000B396A92DBA2D0E942C0E0E2EED2DFE2DFB
:10129000BD960E94260EE02191F0E7E0EA930E94BD
:1012A000BA0BE2E0EA930E94BA0BE2E0EA930E94F2
:1012B000BA0BEBEAF1E0FA93EA930E94E80BED2D0A
:1012C000FE2D7996A92DBA2D0E942C0E0E2EED2DF5
:1012D000FE2DB3960E94260EE02191F0E7E0EA93FE
:1012E0000E94BA0BE2E0EA930E94BA0BE0E0EA93B4
:1012F0000E94BA0BEBEAF1E0FA93EA930E94E80B42
:10130000ED2DFE2D7196A92DBA2D0E942C0E0E2EBC
:10131000ED2DFE2D79960E94260EE02171F0E7E07A
:10132000EA930E94BA0BE2E0EA930E94BA0BE3EB65
:10133000F1E0FA93EA930E94E80BED2DFE2D3A9628
:10134000A92DBA2D0E942C0E0E2EED2DFE2D71967C
:101350000E94260EE02171F0E7E0EA930E94BA0BAA
:10136000E0E0EA930E94BA0BE3EBF1E0FA93EA9330
:101370000E94E80BED2DFE2D3096A92DBA2D0E946E
:10138000200E0E2EED2DFE2D3A960E94260EE02107
:1013900071F0E7E0EA930E94BA0BE4E0EA930E945E
:1013A000BA0BE3EBF1E0FA93EA930E94E80BF59BAA
:1013B0003CC0E0E0EA93E1E0EA930E948E0BE6E0B5
:1013C000EA930E94BA0BE6E0EA930E94BA0BE6E0C9
:1013D000EA930E94BA0BE6E0EA930E94BA0BE6E0B9
:1013E000EA930E94BA0BE6E0EA930E94BA0BECEB98
:1013F000F1E0FA93EA930E94E80BE6E0EA930E9498
:10140000BA0BE6E0EA930E94BA0BE6E0EA930E9488
:10141000BA0BE6E0EA930E94BA0BE6E0EA930E9478
:10142000BA0BE6E0EA930E94BA0BF798E1E0E0938A
:1014300031030E947001A0910C03B0910D031B9722
:1014400054F0E0917A00E064E0937A00E0E0E09309
:101450000C03E0930D031B9926C0E32DF42DE43615
:10146000A0E0FA0719F4E4EFF1E014C0E43FA1E0D2
:10147000FA0719F4E8EEF3E00DC0E83EA3E0FA073E
:1014800019F4E0E1F7E206C0E031A7E2FA0759F407
:10149000E4E6F0E03E2E4F2EF69AECE2F1E0FA930D
:1014A000EA930E94AC0C19992BC0E62DF0E030971E
:1014B00031F4EAE06E2EF79A2C982D9A1BC0EA3090
:1014C000A0E0FA0729F4E4E16E2EF79A2C9A11C0F5
:1014D000E431A0E0FA0731F4EEE16E2EF79A2C9A8F
:1014E0002D9A08C0EE31A0E0FA0751F46624F79A6D
:1014F0002C982D98ECE2F1E0FA93EA930E94AC0C60
:101500001A9917C0E0E0F099E1E0E03019F4F09AA0
:10151000F69A06C0E13069F4F098F69A77248824A8
:10152000ECE2F1E0FA93EA930E94AC0C0E949F0B6C
:10153000F79AE0E0319BE1E00E2EA0E0F599A1E002
:10154000E0E00E94030EE02111F0F59AF79AE0E046
:101550003199E1E00E2EA0E0F599A1E0E1E00E94D2
:10156000030EE02111F0F598F79AA0E01A9BA1E094
:10157000E0E01B9BE1E0EA23C1F0F894E091000376
:10158000F09101036091020370910303ADE0B0E0BC
:101590000E948B0E0E949F0BE8EEF3E0FA93EA9311
:1015A0000E94AC0CF69AF79A7894A0913103A1307E
:1015B00011F00C94520BF894F59B09C0E0910003D4
:1015C000F0910103609102037091030318C0E09150
:1015D0000803F091090360910A0370910B03A09135
:1015E0000003B091010380910203909103030E94D4
:1015F000E40DE72DF82D0E94FE0D0E94DF0DE09313
:101600000403F09305036093060370930703E0E07F
:10161000E0933603E0913703F0913803609139038A
:1016200070913A03A0910403B091050380910603E1
:10163000909107030E94670E0E944C0DA2E3B3E055
:101640000E94E50C0E945B0E5A9A5A98E0E0E093E3
:101650003003A0913003A530E8F45524E8E05E168D
:1016600098F4E0913003F0E0EE5CFC4F1080E52D43
:10167000A1E00E94F60DE12111F4599801C0599A98
:101680005B9A5B985394EACFE0913003EF5FE0936D
:101690003003DFCF59985A9A5A98E0E0E09331032B
:1016A000789483CFD8C9FFCFE881E07111F05D9ABB
:1016B00001C05D98E881E07211F02F9A01C02F9867
:1016C000E881E07411F02E9A01C02E98E881E0784C
:1016D00011F05C9A01C05C9885E08A95F1F75E9AFA
:1016E0008DE08A95F1F75E988DE08A95F1F7C4C098
:1016F000E881EA93D9DFE881E295E883E881EA931B
:10170000D3DF85E88A95F1F7B7C0E981EA93F0DF86
:10171000289AE881EA93ECDF28980FC0E881F0E08E
:10172000E55CFC4FE081A981EA0FEA93E1DFE98102
:10173000E0933F03E881E093400322960895E2E0BE
:10174000EA93D6DFE3E0F0E0FA93EA930E94AC0C70
:10175000ECE0EA93CDDFE1E0EA93CADFE3E0F0E01A
:10176000FA93EA930E94AC0CE0E0E0934003E0932C
:101770003F030895A881AA3031F0E0914103A09180
:101780003F03AE1768F0E0E0EA93E0914003EF5FBB
:10179000E0934003EA93C2DFA881AA3009F46CC049
:1017A000E0913F03EF5FE0933F03289AE881EA93DB
:1017B0009FDF289861C01A93A981BA81ED91A9830E
:1017C000BA831E2FE03019F01A93D4DFF5CF0EC084
:1017D0001A93E981FA813196E983FA833197E4918A
:1017E0001E2FE03019F01A93C5DFF3CF188123962E
:1017F0000895559A279A269A549A569A209A579A53
:101800005E9828985F98E881E0934103E058E09360
:101810003D03E881E054E0933E03E4E1F0E0FA9315
:10182000EA930E94AC0CE0E3EA933EDF88EC90E0A0
:101830000197F1F7E0E3EA9337DF88EC90E0019756
:10184000F1F7E0E3EA9330DF88EC90E00197F1F7FD
:10185000E0E2EA9329DF88EC90E00197F1F7E8E213
:10186000EA9346DFE4E0EA9343DFE5E8EA9340DF0A
:10187000E6E0EA933DDF63DF2196089524971A930B
:101880000A93E0E0FAEC6AE97BE3EA83FB836C838A
:101890007D8300E0AB85AA2392F4E885F9856A850B
:1018A0007B850E94EE0DE887F9876A877B87AE818A
:1018B000BF811196AE83BF831197EDE2EC93EA816D
:1018C000FB816C817D81A885B9858A859B850E9475
:1018D000320E1E2F103071F4003061F4AA81BB81EA
:1018E0008C819D81A130E0E0BE07E0E08E07E0E062
:1018F0009E0751F4AE81BF811196AE83BF831197CD
:10190000E12FE05DEC9301E0EA81FB816C817D8158
:10191000A885B9858A859B850E94570EE887F98737
:101920006A877B87AA81BB818C819D81EAE0F0E098
:1019300060E070E00E94320EEA83FB836C837D835B
:101940000E94AC0E09F0BBCFAE81BF81E0E0EC930A
:10195000198108812C960895E991F991309639F012
:1019600080ED97E00197F1F7A8953197C9F70895B1
:10197000552342F4503811F4E0FF04C03196691F3A
:10198000791F6BF050E8572711F45F9373C05F3FE6
:1019900031F0660F000C57956795752F08955F938A
:1019A00000200AF073C06CC050E8192E1522880F71
:1019B000991F9527550F879550E8072E0522660F2A
:1019C000771F7527550F67950895689401C0E894AF
:1019D0005F93F2DF703818F07F3F08F44BC056E198
:1019E000571BAAF4519558300EF4593030F0EFEFF0
:1019F000FFEF6FEF7FE777F91AC077275523B9F02C
:101A0000EE0FFF1F661F771F5A95D1F710C077277B
:101A1000583028F0EF2FF62F672F5850F9CF552365
:101A200031F076956795F795E7955A95D1F70020AF
:101A30000AF4D4D05F910895689401C0E894309777
:101A400060407040B1F0002426F0772312F4009437
:101A5000C5D0172E7EE1112032F07A95EE0FFF1FD0
:101A6000661F111CF9CFEF2FF62F612D5F938ADFD0
:101A70005F910895EE27FF27662777275F910895E6
:101A8000EFEFFFEF6FE77FEF5F910895EFEFFFEF6D
:101A90006FE77FE75F9108955F9386DF703851F3BA
:101AA000903841F301240894791F23F41CF300209B
:101AB0003AF3ECCF0F921F932F933F934F9311273D
:101AC00022279927689FA0018F9F302D410D591F14
:101AD0006B9F300D411D591F8E9F27D0BF9F25D072
:101AE0006A9F23D0BE9F1DD0AF9F1BD0AE9F110D0C
:101AF000291F391F491F591FE32FF42F652F522F1C
:101B00004F913F912F911F910F9066232AF0550F0F
:101B1000EE1FFF1F661F02C073954BF229DF5F9116
:101B20000895100D211D391F02C0200D311D491FC0
:101B3000591F08955F9338DF703821F411200AF49B
:101B40009FCFA4CF903809F495CF01240894970B28
:101B50001BF4D4F30020F3CF792F1F932F933F93DF
:101B60004F9311241127222733274427552790E22A
:101B7000AE17BF078607410730F0AE1BBF0B860BC1
:101B8000410B089401C08894551F221F331F111C5C
:101B9000AA1FBB1F881F441F9A9551F7F901612D99
:101BA0004F913F912F911F91662332F0550FEE1FF9
:101BB000FF1F661F7A9543F2DBDE5F910895EA0FFF
:101BC000FB1F681F791F0895AE0FBF1F861F971F49
:101BD0000895AE1BBF0B860B970B0895F09560958B
:101BE0007095E195FF4F6F4F7F4F0895EE230E2EB6
:101BF000EA2F19F0EE0F0A94E9F708956F2F660F98
:101C0000660B762F0895EA17E1E009F0EE270895B4
:101C1000EA17FB07E1E00CF4EE270895AE17BF07C3
:101C2000E1E00CF4EE270895AE17BF07E1E00CF0F9
:101C3000EE270895EA17FB07E1E00CF0EE27089580
:101C4000AE17BF07E1E008F4EE270895AE17BF070F
:101C5000E1E008F0EE270895EA17FB07E1E008F05D
:101C6000EE2708953F934F935F9300241124442758
:101C7000552730E2AA0FBB1F881F991F001C111C9B
:101C8000441F551F0E1A1F0A460B570B28F40E0E41
:101C90001F1E461F571F01C0A1603A9559F7FD014D
:101CA000BC01D001CA015F914F913F910895DADFE5
:101CB000FD01BC010895ED93FD936D937C93089510
:101CC0007A936A93FA93EA930895689401C0E8942A
:101CD00001D0B5DE182E862F612D192E972F712D6C
:101CE0001B2EBF2FF12D1A2EAE2FE12D0895129627
:101CF00002D0BF011297119602D0FE2F1197F999C9
:101D0000FECFFF93FFB7F894A1BDB2BDF89AE0B53E
:101D1000FFBFFF91089507D012960F01FB0103D07A
:101D2000F0011297089507D01196EF93EF2F03D08B
:101D3000EF9111970895F99B02C0A895FCCF9FB72A
:101D4000F894A1BDB2BDF89A80B5E81719F0E0BDCE
:101D5000FA9AF99A9FBF08953097604070400895AD
:00000001FF
